:020000040000FA
:020000002C28AA
:040002000034003492
:0800080009007228E737613995
:10001000BA364C10E737E3347238E237A032612247
:10002000653A201D201031102E1C3218321731185D
:10003000A01B652B7339EF343A3732103417001098
:10004000F520683AF237201D4810E932653720392B
:08005000F5256C34E1366E3732
:0800580051280F398207192A13
:10006000212A272A2E2A362A3F2A452A4C2A542A70
:100070005D2A632A6C2A742A7D2A842A8D2A0F39E4
:100080008207FF34FF34FF34FF34FF34FF34FF3482
:10009000FF34E734D034B834A1348A3472345B345A
:1000A0005B342F233E218316FF2390008312A3018C
:1000B000A401A901AA01AB01AC01AD01AE01AF01E0
:1000C000B001B201B4010730B600FE30B800BA0189
:1000D000B9010030BB00BC01BD01BE01C0019422CA
:1000E000D7218312851D2D140510051105124623F5
:1000F00005140515051648231423051405150516C2
:100100004823962196219621962105100511051266
:100110006221ED222D1C9B28831285199B288519AD
:100120009A2805100511051240230514051505161A
:1001300040238F289E220510051105128312851D6C
:100140009B284623051405150516A8217A21B02100
:1001500083128519B228A901A821831205162D142E
:10016000AC01B5280430AE00AD01AF08031DBB28BB
:10017000AE0BBB282D29AA08031DD528AB08031DEB
:10018000D128831229180512F4222D18D828321CE0
:10019000D8284E30AA00AB00291483120512A821DA
:1001A000D82883120516AB03D82883120512AA0398
:1001B0003008B10030108130A318A430231CA530C2
:1001C000831699003C238312191B7321B0108E30C3
:1001D000A3188630231C8930831699003C23831290
:1001E000191F7621B0113012231C08298530A3185D
:1001F000A630831699003C238312191BB0158A3050
:10020000A3188230831699003C238312191F3016DD
:1002100030083106031DA821B21C2029321C2029D8
:100220002F182029AF1820292F192029301AB0148F
:10023000B0193014B018202930182029B014301407
:100240008312301825290514262905108312B018A9
:100250002B2905152C290511A6289422D721231C0A
:100260003529A31C3829A30139292314A3103929BE
:10027000A3149621851D3929ED22A6288312850114
:1002800053218316813099008316813081008312B7
:1002900081010730831290000E08A6000F08A70006
:1002A000A401A80108008312043099002A308316A3
:1002B0008500831208002B30831685000E308312D0
:1002C00099003C2B2830831685008312402385102B
:1002D000402385144023851040232A30831685004F
:1002E00083124023080030142C140800B0142C187A
:1002F000AC14080083120508B7000B198A293918B5
:100300007D290108380203187D29051405150516F5
:1003100039147D290B11370815398500B90183126D
:100320000C1C94290C109429AF0A080083120514A0
:10033000051523180512A31CA1290511341C05104D
:10034000A22905104923051405150516492308009F
:10035000BB1C0800BC019430BD000430BE00080086
:10036000BB1C0800BC0B0800BD0B0800BE0B08003E
:1003700083120514051505168312003099008316A3
:100380009901093085008312851085128316961510
:100390008B156300000083120508831696110B105D
:1003A0008B118B10831285145321ED22A8298312FF
:1003B0000508B7005B2138230730B6005B233608F9
:1003C0008038831699003C238312191BED29360AC5
:1003D0000F3C0319ED29B60ADE29F3215321370812
:1003E00015398500080036083F20B8000800B30121
:1003F0005B2138238A30831699003C238312191B12
:100400000D2A53218312023099000B308316850088
:1004100083128516382335082D2853210800B3038D
:10042000330FB3032A3083168500831204309900FA
:100430000800000000000000191F102AB30F192A3D
:100440000F2A3F23191F102AB30F212A0F2A3F23F7
:100450000000191F102AB30F272A0F2A3F2300007C
:100460000000191F102AB30F2E2A0F2A3F23000065
:1004700000000000191F102AB30F362A0F2A3E234E
:10048000191F102AB30F3F2A0F2A3E230000191FFD
:10049000102AB30F452A0F2A3E2300000000191F1F
:1004A000102AB30F4C2A0F2A3E2300000000000040
:1004B000191F102AB30F542A0F2A3D23191F102A7F
:1004C000B30F5D2A0F2A3F233F233F230000191F4C
:1004D000102AB30F632A0F2A3D2300000000191FC2
:1004E000102AB30F6C2A0F2A3D23000000000000E1
:1004F000191F102AB30F742A0F2A3C230000191F5A
:10050000102AB30F742A0F2A3C23000000000000B9
:10051000191F102AB30F742A0F2A3B230000191F3A
:10052000102AB30F742A0F2AC0223123F721B401F5
:10053000B022330203183414ED2208004623B5011B
:100540003508F039031DAE2A4323F7213308193E3D
:10055000031CAC2AB50AA02ACE22DF22ED22080015
:10056000831601309B001C141A0883120319BE2A3B
:10057000C10041090319BE2A41080800963008004D
:10058000831602309B001C141A088312B50035092B
:100590000319CB2A08000E30B5000800831601307D
:1005A0009B0033089A001C1555309D00AA309D0011
:1005B0009C141C1183128C1FDB2A8C1308008316D9
:1005C00002309B0035089A001C1555309D00AA305A
:1005D0009D009C141C118312DB2A0E08A6000F0834
:1005E000A7002408A8000800B2103218B214321074
:1005F00083120E08A5002602031D32142508A6004A
:100600000F08A5002702031D32142508A70024089F
:100610002802031D32142408A8003218122BAC1C27
:1006200008003214AC0108000230192304301923E9
:100630000800C100051605150514492341180512C7
:10064000C11805114119051046230800A0002830E3
:10065000A1003123A10B292BA00B272B080064300C
:10066000262B3823382338233823382338233823BC
:100670003F233F233F233F233F233F233F230800C4
:100680003230A2004A2B6430A2004A2B492349236E
:100690004923FA30A2007A21A20B4B2B08008312C7
:1006A0000518572B00000514000005100800051060
:1006B00000000514080083120519632B00000515BE
:1006C000000005110800051100000515080083123F
:1006D0000519722B00000515000000000000000045
:1006E00005110800051100000000000000000515BC
:1006F00008008312051A812B000005160000051260
:10070000080005120000051608008312051A902B38
:10071000000005160000000000000000051208009F
:0E072000051200000000000000000516080091
:02400E00943FDD
:00000001FF
